:10000000B6EF01F00000000000EF00F0000000007B
:0A0010000000000000000000F3D71C
:0A001C00530E0D6E0D2EFED71200DC
:10002600240E0C6EB50E0D6E0D2EFED70C2EFCD7C3
:06003600000000001200B2
:0C003C00000000000000000000001200A6
:100048000001BEBF02D08B9601D08B86BEBD02D008
:100058008B9401D08B84BEBB02D08B9201D08B8253
:10006800BEB902D08B9001D08B8080B102D0898834
:1000780001D08998898ADEDF899ABEB702D08B962B
:1000880001D08B86BEB502D08B9401D08B84BEB3D1
:1000980002D08B9201D08B82BEB102D08B9001D05E
:1000A8008B8080B102D0898801D08998898AC2DF83
:0E00B800899A80A102D0B3DF01D0ACDF120024
:1000C6000001BB51010A03E1800EBB6F14D0BB5186
:1000D600020A03E1C00EBB6F0ED0BB51030A03E157
:1000E600940EBB6F08D0BB51040A03E1D40EBB6F5C
:1000F60002D0800EBB6FBC05006EBB51002600C04F
:10010600BBF0808100C0BEF09CDF8091BDC0BEF018
:0601160098DF8081120059
:0E011C0000018091BBC0BEF091DF8081120017
:0E012A00000E9EBA010E016E01C000F0120020
:10013800AECF02F0ABA202D0AB98AB8802C001F000
:0601480001C000F01200EE
:10014E005B6A5B500001B75D18E35B50B825E16E4A
:10015E00000EB921E26E5B50B625006E150EE96EEB
:10016E00000EEA6E0050E926D8B0EA2AEECFE6FF7E
:10017E005B50B71902E05B2AE4D7B751B825E16EA0
:0C018E00000EB921E26E000EE66E1200B9
:10019A000001B651010A03E1800EB66F14D0B651C0
:1001AA00020A03E1C00EB66F0ED0B651030A03E18C
:1001BA00940EB66F08D0B651040A03E1D40EB66F96
:1001CA0002D0800EB66FB705006EB651002600C089
:1001DA00B6F000C0BEF033DF8091BA6BBA51B825D1
:1001EA00E96E000EB921EA6EEE50000A0BE0BA5130
:1001FA00B825E96E000EB921EA6EEECFBBF089DFB1
:08020A00BA2BECD78081120031
:10021200929A92989490949294949496899A8998A6
:100222008B968B948B928B90FDDEFCDEFBDE8B82B9
:100232008B80898A02DF899AF5DE898AFEDE899AB5
:10024200F1DE898AFADE899AEDDE8B90898AF5DE03
:10025200899AE8DE898AF1DE899A8B928B86898A6D
:10026200ECDE899ADFDE8B968B80898AE6DE899ABC
:100272008B90898AE2DE899AD5DE898ADEDE899AC6
:100282008B80898ADADE899ACDDE8B90898AD5DEE7
:10029200899A8B868B848B828B80898ACEDE899A1F
:0802A200C1DE000180811200A1
:1002AA003FDF0050010AFCE142DF00C0B6F0B6C0F1
:0402BA0000F012003E
:1002BE00400E0001BE6FC1DEB86BD40EB825F66ECF
:1002CE00070EF76E000EF722000EF86E000EF822E3
:1002DE000900F5CFBBF01BDFB851070A02E0B82BBF
:1002EE00ECD7020EBE6FA9DEB6C0BBF0B7C0BCF035
:0602FE00BD6BE2DE120000
:10030400FF0E0001856FFF0E866FFF0E876FFF0ED5
:10031400886F380E816F010E826F000E836F000E9E
:10032400846F2A0E946F010E956F000E966F000E67
:10033400976FFF0E576EFF0E586E000E596E000E2B
:100344005A6EAC8A900EAB6E948E949C9EAA03D087
:08035400AECF00F0FBD7120050
:10035C000900F5CFE6FF0006FBE10106F9E112000A
:10036C000F0EC16E949A94989386938A200E6F6E9A
:10037C00520E706E450E716E430E726E450E736E9C
:10038C00500E746E540E756E490E766E4F0E776E5F
:10039C004E0E786E200E796E470E7A6E500E7B6E76
:1003AC00530E7C6E200E7D6E200E7E6E7F6A460E86
:1003BC005E6E490E5F6E580E606E200E616E330ECF
:1003CC00626E440E636E200E646E700E656E610E6E
:1003DC00666E720E676E200E686E4C0E696E450E60
:1003EC006A6E440E6B6E730E6C6E200E6D6E6E6AC2
:1003FC000ADF010EBE6F22DE0C0EBE6F1FDE010E79
:10040C00B66F010EB76F6F0EB86F000EB96FBFDE0F
:10041C00020EB66F010EB76F5E0EB86F000EB96F9D
:10042C00B6DE8B888B8A4D0E0B6E190E0C6E4F0E32
:10043C000D6E0D2EFED70C2EFCD70B2EFAD700000E
:10044C00000081A608D0B886020EB06E080EAF6E02
:10045C00AC8452DF09D081B607D0B886040EB06EDA
:10046C00110EAF6EAC8448DF030E0B6E8A0E0C6E51
:10047C00550E0D6E0D2EFED70C2EFCD70B2EFAD76B
:10048C0000000000310E5D6E010E5C6E08DF00C0D6
:10049C005BF00050240A01E0F9D75B6A150E0001ED
:1004AC00B46F000EB56F5B50B427D8B0B52BF7DE28
:1004BC00B4C0E1FFB5C0E2FF00C0E6FF150EE96E67
:1004CC00000EEA6E5B50E926D8B0EA2AEE502A0AF2
:1004DC0002E15B6A01D05B2A5B50000AFF0ED8A4D4
:1004EC00000E016E5B504B0AFF0ED8A4000E006E7E
:1004FC000150001201E1D2D75C50010AD8A4DCD023
:10050C001750470AFF0ED8A4000E016E1850530A5C
:10051C00FF0ED8A4000E006E005001161950410AAF
:10052C00FF0ED8A4000E006E01500016D8B4C4D033
:10053C001DC05DF01D50330A2FE1010E0001B66F96
:10054C00010EB76F2A0EA36F2A0EA46F2A0EA56F89
:10055C00200EA66F4D0EA76F6F0EA86F640EA96FBD
:10056C00650EAA6F200EAB6F330EAC6F440EAD6FE1
:10057C00200EAE6F2A0EAF6F2A0EB06F2A0EB16F1F
:10058C00200EB26FB36BA30EB86F000EB96FFFDD08
:10059C008B888B9A020E5C6E5D50320A30E1000142
:1005AC00010EBE6F4BDD010EB66F010EB76F2A0E3A
:1005BC00A36F2A0EA46F2A0EA56F200EA66F4D0EE8
:1005CC00A76F6F0EA86F640EA96F650EAA6F200E31
:1005DC00AB6F320EAC6F440EAD6F200EAE6F2A0EA9
:1005EC00AF6F2A0EB06F2A0EB16F200EB26FB36BC5
:1005FC00A30EB86F000EB96FCADD8B8A8B985D5055
:10060C00310A5AE10001010EBE6F18DD010EB66F02
:10061C00010EB76F200EA36F410EA46F740EA56F61
:10062C00740EA66F650EA76F6E0EA86F740EA96F71
:10063C00650EAA6F200EAB6F740EAC6F720EAD6FA1
:10064C00610EAE6F6D0EAF6F650EB06F730EB16F46
:10065C00200EB26FB36BA30EB86F000EB96F97DD9F
:10066C00020EB66F010EB76F200EA36F200EA46F93
:10067C004E0EA56F4D0EA66F450EA76F410EA86FBF
:10068C00200EA96F760EAA6F610EAB6F6C0EAC6F5D
:10069C00690EAD6F640EAE6F650EAF6F730EB06FFB
:1006AC00200EB16F200EB26FB36BA30EB86F000E9D
:1006BC00B96F6DDD8B988B9A5C50020AD8A482D0EE
:1006CC001750470AFF0ED8A4000E016E1850470AA7
:1006DC00FF0ED8A4000E006E005001161950410AEE
:1006EC00FF0ED8A4000E006E015000166BE0010E38
:1006FC005C6E81AA14D000012D0EB66F020EB76F7E
:10070C00980EB86F000EB96F1CDD300EB66F040E6C
:10071C00B76F890EB86F000EB96F13DD15D081BAA3
:10072C0013D00001280EB66F020EB76F980EB86F7B
:10073C00000EB96F06DD2B0EB66F040EB76F890E67
:10074C00B86F000EB96FFDDC0001020EB66F010E22
:10075C00B76F530EA36F410EA46F540EA56F3A0ED4
:10076C00A66FA76BA30EB86F000EB96F10DD020E4B
:10077C00B66F050EB76F980EB86F000EB96F07DD28
:10078C00020EB66F080EB76F480EA36F440EA46F1F
:10079C004F0EA56F500EA66F3A0EA76FA86BA30E47
:1007AC00B86F000EB96FF3DC020EB66F0D0EB76F9B
:1007BC00890EB86F000EB96FEADC020EB66F0E0E22
:0807CC00B76F77DD63D6FFD79C
:0807D40000000000000C040805
:020000040030CA
:0D000100021F1EFF8381FF0FC00FE00F40A4
:00000001FF
